:10000000C828083035190130A300A201380884003F
:10001000360849203608800484130005FF3E351D4C
:10002000A20C3519A20D32305D20A30B082822083E
:100030000314C328A200083035190130A300A20C14
:1000400038088400360849203608031880043C30FC
:100050005D2036088004A30B1F280314C328B51C99
:10006000C3283528B500351CC32838088400360855
:1000700049200130A100F4305E20360880040130B0
:10008000A100F4305E2829080319C328BE20A90363
:100090004328FF3A80054C2884178005C32883161F
:1000A0009B001C141A08C3288316F83881050F39E1
:1000B000810463000F308104C328A101E83EA00041
:1000C000A109FC30031C6728A00703186428A007B7
:1000D0000000A10F642820186D28A01C71280000C2
:1000E00071280800013EA7000A30A200A3018C205D
:1000F000A70B7728240808000310A00DA10DFF3ED0
:1001000003187C282008C3280310A10CA00CFF3E74
:10011000031884282008C328A501A4011030A600D4
:10012000210DA40DA50D2208A4022308031C230FF2
:10013000A5020318A2282208A40723080318230FE6
:10014000A5070310A00DA10DA60B90282008C32819
:100150001030A800A101A001A70CA60C031CB62812
:100160002208A00723080318230FA107A10CA00C45
:10017000A50CA40CA80BAC282408C32884003108C3
:100180008A003008820083130313831200000800E2
:100190000730990083169F0185018312850185141C
:1001A0002130C500EA23A930C500EA230630C50086
:1001B000EA231330C500EA232030C500EA23EB21EF
:1001C0001C220C30C500851DE7280D30C500EA2330
:1001D0000530B8000430B60001303220CC301A208F
:1001E000BE301A202F200530B8000430B600003091
:1001F00032200120BE000120BF000430A9000130E0
:10020000B000B10143200120C4000120C3002F2011
:100210004110BF1F17293E09B2003F09B30001304A
:100220003207BE0033080318013EBF0041143E08E8
:10023000A0003F08A10004308720C8000F303E0511
:10024000C9004908A600A7017130A2000230A3002E
:10025000A820BE002508BF000530B8000430B60055
:1002600001303220CC301A2044301A202F208C301C
:10027000C500EA234330C500EA2364304802031C6A
:1002800045290130C200F2214C290A30C200411C2C
:100290004B290B30C200F2214808A000A101013017
:1002A0007220C200F2214808A000A1010030722093
:1002B000C200F2210C30C200F2213E08A0003F082B
:1002C000A10003307220C200F221B721FF30BA0032
:1002D000FF30BB00FF30BC00FF30BD0021304802C2
:1002E000031C73299E294808203CC8000130CB001C
:1002F0004B084802031C80290310BA0DCB0F782944
:100300000930CB004B084802031C8A290310BB0D9F
:10031000CB0F82291130CB004B084802031C9429D3
:100320000310BC0DCB0F8C291930CB004B084802B1
:10033000031C9E290310BD0DCB0F9629CB01043061
:100340004B020318AC29AF214B083A3E8400000849
:10035000C500EB23CB0F9F2906305420E128CC3079
:10036000C500EA2341304B07C500EA230800C60157
:10037000411CBC290430C600BF30C500EA2343300D
:10038000C500EA234608C500EB234608C500EB2359
:10039000411CCC290130C600BD30C500EA234230E3
:1003A000C500EA234608C500EB234608C500EB2339
:1003B0000130C600411CDE294130C600BD30C500F9
:1003C000EA234030C500EA234608C500EB2346086F
:1003D000C500EB2308008030C500EA234030C5008B
:1003E000EA2308004208A600A7010530A200A301E5
:1003F000A820C7000130C000063040020318072AB9
:1004000047084F20C500EB23C70AC00FFC29C501D0
:04041000EB230800D2
:100438004130CB0080304B020318282A4B084F204C
:10044800C500EB23CB0F1E2ACB01C3304B02031888
:10045800FE2A4B08C23C031CFB2A3422C500FB2A97
:1004680002308A004B0882070134A1341134513418
:10047800A1340134E13411341134E13401348134CC
:10048800413441344134813401340134013401347C
:10049800FF34FF3400340034FF3400342134203476
:1004A8003C3423340634393460348034A334BD34C6
:1004B8002B342D3433348034FF340034003400348A
:1004C80000340F340F340F34003400340034033454
:1004D80007340F340D340D340D34053400340F3423
:1004E8000F340F3400340F340F340F3400340F340A
:1004F8000F340F3400343F343F343F3404340F3466
:100508000F34073400340C340C3400340034003415
:1005180004348434453445348434043484344534D0
:10052800453484340034FF34003400340034FF345C
:100538000034843404340034FF34FF34003400348D
:100548000034E134F23412341234123412341234D6
:100558001234123412341234123412341334133461
:1005680013341034103408340434023401340134A0
:1005780001340134013401340134013401340134CB
:1005880001340134013401340134013401340134BB
:10059800013401340134813481348134013401342B
:1005A800013401340134013401340134013401349B
:1005B800FE34003400340034103414341634153446
:1005C8001434103413341434143413340034FF3412
:1005D800003400340034FF34003410341034003454
:1005E800FF34FF34003400340034FF34FF34EB238D
:1005F800CB0F292AC5010130CB0029304B02031843
:10060800082BEB23CB0F012BCB01CE304B02031869
:10061800E92B4B08CD3C031CE62B1423C500E62B25
:1006280003308A004B088207033402340334003451
:1006380000343E34413441344134233400340034EE
:100648000034FF3400340034003440344034403443
:1006580041345F3440344E34513451344E340034D4
:10066800FF34003400340034FF3400344234403462
:100678000034FF34FF3400344034C0344734473446
:100688004634863406340634063406340634863452
:10069800C634063486344634463486340634463402
:1006A800C6344634463486340634863446344634B2
:1006B8008634063486344634463486340634063462
:1006C8000634863446348634063406340634063412
:1006D80006344634C6344634463486340634463402
:1006E8000634063406340634023401348034C03407
:1006F8000034803440344034803400344034C034D2
:1007080040344034C0340034FF3400340034003402
:10071800FF340034083400340034FF34FF348034AC
:1007280090349F349034903490348F3480349234A1
:1007380095348934803480349F3480348D349234B5
:1007480092348D34803490349F34923492348D3482
:100758008034983494349234993480348F3490347B
:1007680090348F348034803480348E349134923491
:100778008D34933480348034803490349F34923470
:100788008234813480349F3480348E34913491346F
:100798008A34803480349F3480349834943492344A
:1007A8009934803490349F349234823480349E3427
:1007B800BF34BF34BF34BF34BF349E348134813436
:1007C8008034FF34EB23CB0F092B080005100130D0
:1007D800CA0009304A020318FB2BC51B0516C51FA2
:1007E80005120310C50D85168512CA0FED2B0514C9
:0607F80008006300FD2B68
:02400E00CC3FA5
:104200003E005100490045003E00000042007F0092
:1042100040000000420061005100490046002100BA
:10422000410045004B0031001800140012007F00CF
:104230001000270045004500450039003C004A00B9
:104240004900490030000100710009000500030029
:10425000360049004900490036000600490049007F
:1042600029001E00080008003E00080008000800A1
:10427000080008000800080000006000600000005E
:104280000000FF0001000100E10011008900490069
:104290004900C90049000900C90049004900090056
:1042A0000900090009001100E100010019001900CE
:1042B0001900F900F900F90019001900190081002E
:1042C000C100E1002100E100E100C1000100E100C6
:1042D000E100E1004100E100E100C1006100E10016
:1042E000E100C1000100E100E100E1004100E10066
:1042F000E100C10001000100010001000100010016
:00000001FF
